:100000000C9462000C944F1A0C947C1A0C948A0085
:100010000C948A000C948A000C948A000C948A0038
:100020000C948A000C948A000C948A000C948A0028
:100030000C948A000C94C2060C948A000C948A00DA
:100040000C94A91A0C948A000C94FC1D0C94371E75
:100050000C948A000C948A000C948A000C948A00F8
:100060000C9446050C948A00000000002400270030
:100070002A0000000000250028002B0000000000DE
:1000800023002600290004040404040404040202DA
:100090000202020203030303030301020408102007
:1000A0004080010204081020010204081020000012
:1000B0000007000201000003040600000000000029
:1000C0000000DF1F11241FBECFEFD8E0DEBFCDBF81
:1000D00012E0A0E0B1E0E4ECF1E402C005900D9282
:1000E000A63BB107D9F714E0A6EBB2E001C01D9220
:1000F000AF39B107E1F710E0C4ECD0E004C02297BB
:10010000FE010E94DC20C23CD107C9F70E942420D6
:100110000C94E0200C940000FB01DC0102C0019073
:100120000D9241505040D8F708958091B602813029
:1001300019F482E08093B6028091B602833019F4FC
:1001400084E08093B6020895E3E0F0E089E08093D4
:100150005700849190E08670863009F491E0892FF1
:1001600008951F93182F0E94A400882379F09FB749
:1001700081E08093E503F894A89588E1809360007E
:1001800010936000112309F0A8959FBF1F91089557
:10019000382F20E08091E6039091E7038227932790
:1001A00040E061E270E19C01220F331F97FF04C021
:1001B000C9018627972701C0C9014F5F483099F7C9
:1001C0009093E7038093E60308958436910520F425
:1001D000BC0180E090E025C08E3B910550F48A552B
:1001E0009040BC0180E090E02AE030E040E050E048
:1001F00016C0823D910550F4845B9040BC0180E0C4
:1002000090E024E630E040E050E009C08D5C904092
:10021000BC0180E090E028E532E040E050E00E9440
:10022000332024E630E040E050E00E94332008957F
:1002300090E08C599F4F0E94E5000895DC0198964C
:10024000EC91F0E0E770F070E256FD4F8081089588
:10025000FC0120A530E0C9018170907001962770E3
:10026000307035952795820F931F880F880F08955A
:100270008F929F92AF92BF92CF92DF92EF92FF92B6
:100280000F931F938C010E941E01D80197962C9109
:1002900030E043E150E0249FF001259FF00D349FB2
:1002A000F00D1124E251FE4F80809180A280B38036
:1002B00090E00F96AA2797FDA095BA2FBC01CD011B
:1002C00020E43FE14DE750E00E943320A501940176
:1002D0000E94662069017A0180ED97E0A0E0B0E01D
:1002E000C80ED91EEA1EFB1ED80198968C91887103
:1002F00081F060E07EEE8AEB9BE0A50194010E9414
:10030000662028513C4F4F4F5F4FC20ED31EE41E54
:10031000F51E87EE93E0A0E0B0E0C80ED91EEA1EFD
:10032000FB1EC701B60128EE33E040E050E00E941A
:100330006620CA01B90128EE33E040E050E00E9497
:1003400033201F910F91FF90EF90DF90CF90BF90DF
:10035000AF909F908F9008951F93182FDB01FA01A3
:10036000482F469530E0848190E083709070982FFC
:1003700088272081820F911D11969C938E938481F2
:1003800090E08C70907076E0880F991F7A95E1F775
:100390002181820F911D13969C938E9312978481D5
:1003A00090E08073907064E0880F991F6A95E1F780
:1003B0002281820F911D15969C938E9314978481B0
:1003C00090E0807C9070880F991F880F991F23817F
:1003D000820F911D17969C938E93169735961896BB
:1003E0003F5F431708F0BFCF10FF50C08081829558
:1003F00086958695837090E02DE431E0AC01429FB4
:10040000C001439F900D529F900D11240C961196A0
:100410009C938E93808190E044E0969587954A95D1
:10042000E1F783709070AC01429FC001439F900D33
:10043000529F900D11240C9613969C938E931297B5
:10044000808190E0969587959695879583709070BA
:10045000AC01429FC001439F900D529F900D11240B
:100460000C9615969C938E931497808190E08370E0
:100470009070AC01429FC001439F900D529F900D20
:1004800011240C9617969C938E9316971F9108959E
:1004900023E08032920718F420E030E026C023E009
:1004A000883E920748F49C012F51334054E0369522
:1004B00027955A95E1F719C027E0803D920720F46F
:1004C0009C012C5D334011C028E08839920718F058
:1004D0002FEF33E00AC09C01285C374044E036959A
:1004E00027954A95E1F72D503C4FC90108958C306E
:1004F000910548F49C0174E0220F331F7A95E1F7CF
:10050000285D3C4F17C023E0843F920720F49C01F4
:1005100024523C4F0FC024E08030920718F020E9AD
:1005200038E008C09C012657334F64E0220F331F88
:100530006A95E1F7C90108959C01369527952575BF
:100540003575821B930B9C0136952795369527951B
:100550002373337383739373280F391FC901E4E046
:1005600096958795EA95E1F7820F931F8F709F709C
:1005700021E031E0AC01429FC001439F900D529FAA
:10058000900D1124892F0895882339F02D980000AB
:100590002B9A00002D9A000008952D9800002B98AA
:1005A00000002D9A000008952D9A000083B12D9827
:1005B000000090E0B4E096958795BA95E1F78170D8
:1005C00008950F931F93082F5C9A2D985C9810E064
:1005D000802F80780E94C402000F1F5F1830C1F77F
:1005E0002D981F910F9108958F770E94E102089531
:1005F0000F931F93082F10E0802F80780E94C40271
:10060000000F1F5F1830C1F72D981F910F910895AB
:100610000F931F932D9880E000E0182F110F0E9478
:10062000D402810F0F5F0830C1F71F910F91089519
:100630000E94F4020E9408035C9A08951F93162FEB
:1006400080680E94E102812F0E94F8025C9A1F914B
:1006500008951F931091DB021827E2EDF2E0E80FF6
:10066000F11D89E767850E941E038DE3612F0E94BB
:100670001E0382E4612F0E941E031F91089586E2EB
:100680000E94180308950F931F938BE20E94180392
:10069000082F8CE20E941803282F30E096E0369550
:1006A00027959A95E1F710E0000F111F000F111F19
:1006B000202B312BC9011F910F9108950F931F9388
:1006C0008C018CE1F80164810E941E038DE1F80128
:1006D00065810E941E038EE1F80166810E941E035F
:1006E00080E2F80167810E941E0381E2F8016085C3
:1006F0000E941E0382E2F80161850E941E0383E2CC
:10070000F80162850E941E0384E2F80163850E945D
:100710001E0385E2F80164850E941E038AE2F80147
:1007200065850E941E038EE6F80166850E941E0301
:100730008FE6F80167850E941E0380E7F801608953
:100740000E941E0381E7F80161890E941E0382E76F
:10075000F80162890E941E031F910F910895EF9284
:10076000FF920F931F93CF93DF937B018C01603037
:1007700028E372072CE982072CE1920728F520E88C
:1007800036E948E950E00E946620E9016897B9011E
:1007900080E090E020E839E647E65FEF0E943320F2
:1007A0006E0D7F1D801F911F32E0660F771F881F1F
:1007B000991F3A95D1F721E732E040E050E00E94DE
:1007C0006620890180E421C020E03DE241E351E060
:1007D0000E946620E9016897B90180E090E020E07E
:1007E00033ED4EEC5EEF0E9433206E0D7F1D801FB7
:1007F000911F660F771F881F991F21E732E040E0A5
:1008000050E00E946620890180E69E012F71622FD0
:10081000680F85E70E941E0386E7612F0E941E0372
:1008200087E7602F0E941E03CDB7DEB7E6E00C9489
:10083000CB209F92AF92BF92CF92DF920F93DF9324
:10084000CF9300D000D0CDB7DEB7982E83E00E94C2
:1008500018038093FB0284E00E9418038093FC023B
:1008600086E060E00E941E0387E061E00E941E03B4
:1008700089E06FE70E941E038AE065E00E941E0384
:100880008BE062E10E941E038CE065E10E941E0382
:100890008DE06DEF0E941E038EE060E00E941E035B
:1008A000992019F08DE492E008C08091F90223E1CB
:1008B000829FC001112482519E4F0E945E0380E3FB
:1008C0006CE80E941E0382E36FE00E941E0383E334
:1008D00062E40E941E0384E36AE00E941E0385E333
:1008E0006AE20E941E0386E36DE20E941E0387E314
:1008F00064ED0E941E0388E360E00E941E0389E30A
:1009000060E00E941E03992049F065E8A62E61EC84
:10091000B62E61ECC62E6EEDD62E08C0A090DB027E
:10092000B090DC02C090DD02D090DE020AE38D2D93
:100930009927AA27BB2789839A83AB83BC83802FFF
:1009400069810E941E03802F8B5F69810E941E03B4
:10095000DC2CCB2CBA2CAA240F5F0E3341F783E496
:100960006FEF0E941E0384E46FEF0E941E0385E474
:100970006FEF0E941E0386E46FEF0E941E03992012
:1009800019F08DE666E003C08DE66091DF020E94FB
:100990001E0389E760E00E941E038AE76091E0027F
:1009A0000E941E0383E760E00E941E0384E760E06C
:1009B0000E941E03992029F060EC7AEC89E896E306
:1009C00008C06091D7027091D8028091D9029091AD
:1009D000DA020E94AF030F900F900F900F90CF910B
:1009E000DF910F91DF90CF90BF90AF909F900895CF
:1009F00087E061E00E941E038EE764E20E941E030E
:100A000088E063E00E941E0388E060E00E941E030D
:100A100087E065E00E941E0385E062E00E941E03FD
:100A200083E00E9418038093FB0284E00E94180375
:100A30008093FC02089590E0411191E0880F982B7B
:100A40009093BA00660F6093BD0030930203209329
:100A500001030895882311F085EC01C085E8809397
:100A6000BC00089585ED8093BC008091BC0084FD9E
:100A7000FCCF089585EC8093BC000895ECEBF0E08A
:100A8000108285E480831092070308951F920F92CD
:100A90000FB60F9211242F933F934F935F936F9351
:100AA0007F938F939F93AF93BF93EF93FF93DF93C6
:100AB000CF930F92CDB7DEB78091B90090E0887FD9
:100AC00090708036910509F4EAC081369105CCF525
:100AD0008832910509F47CC089329105B4F48031E3
:100AE000910509F470C0813191053CF4009709F437
:100AF0000EC1089709F00DC166C08831910509F44F
:100B000067C0809709F005C177C08034910509F46A
:100B100090C08134910544F48033910509F46EC08E
:100B2000C89709F0F6C06CC08035910509F471C012
:100B30008835910509F483C08834910509F0E9C02E
:100B4000A5C08839910509F4DCC089399105ECF418
:100B50008837910509F4A3C0893791054CF488368C
:100B6000910509F49CC08037910509F0D2C097C067
:100B70008838910509F4C5C08039910509F492C0FF
:100B80008038910509F0C5C08DC0803B910509F4FE
:100B9000A5C0813B91054CF4803A910509F499C0B8
:100BA000883A910509F0B5C099C0803C910509F4D7
:100BB000AAC0883C910509F4A6C0883B910509F0BC
:100BC000A8C080E08CC0809103038093BB009BC0D1
:100BD000809106038150809306038F5F09F43FC024
:100BE000E0910403F091050381918093BB00F093A1
:100BF0000503E093040387C082E049C083E047C057
:100C000084E080930803809107038B7F8093070320
:100C100062C08091BB00E0910403F09105038193D1
:100C2000F0930503E09304038091060381508093C1
:100C3000060380910603823008F065C062C080918F
:100C4000BB00E0910403F09105038193F093050349
:100C5000E093040380910603815080930603809102
:100C600007038B7F809307038091070380FF4FC0AA
:100C7000809107038E7F8093070380910703826032
:100C80008093070384EA8093BC0043C085E080938F
:100C90000803809107038B7F8093070338C010926D
:100CA000060331C0E0910103F0910203309749F14E
:100CB0009091BB00809106038F5F80930603815063
:100CC00011F060E001C062E09983CE0101960995C0
:100CD0001BC00E9432050E943A051BC081E0E091D2
:100CE0000103F0910203309761F0882311F461E071
:100CF00001C063E0CE010196099599819093BB00F4
:100D000003C080E001C081E00E942A0502C00E9469
:100D100032050F90CF91DF91FF91EF91BF91AF918D
:100D20009F918F917F916F915F914F913F912F9103
:100D30000F900FBE0F901F90189525B190E0FC0109
:100D4000EE0FFF1FE80FF91FE359FC4F8081282B9E
:100D500025B988B19181892B88B98BB19281892B72
:100D60008BB9089585B190919D03892385B988B188
:100D700090919E03892388B98BB190919F03892319
:100D80008BB908951F920F920FB60F9211241F93E3
:100D90002F933F934F935F936F937F938F939F9383
:100DA000AF93BF93CF93DF93EF93FF9310914003E3
:100DB00080918402C0918202D0918302181708F0BA
:100DC0005BC08091A0039091A103909387008093D2
:100DD0008600E12FF0E0EE0FFF1FE05AFD4F80810B
:100DE00091810E947702880F991F9093A1038093AD
:100DF000A0038091A0039091A1039E01281B390BB1
:100E0000C90130938302209382022091CD02309158
:100E1000CE02220F331F8217930720F430938302F0
:100E20002093820280914203882339F48091C50285
:100E300080FF59C0183008F456C08FEF9FEF909391
:100E4000890080938800809184009091850080972C
:100E5000D0F30E94B20680914103882339F4809137
:100E60004003882319F081500E949D068091400321
:100E70008F5F809340033EC08091A0039091A103B7
:100E80009093870080938600D093A103C093A00322
:100E900080914203882319F08FEF9FEF06C0809165
:100EA000A0039091A103885592409093890080936C
:100EB000880080E49CE99093830280938202809171
:100EC0008400909185008097D0F30E94B2068091B3
:100ED0004103882329F48091840281500E949D0659
:100EE0001092400307C08091A0039091A103885500
:100EF0009240A5CFFF91EF91DF91CF91BF91AF913C
:100F00009F918F917F916F915F914F913F912F9121
:100F10001F910F900FBE0F901F90189590E0880FB3
:100F2000991F880F991F8C30910518F42CE030E040
:100F300007C09C0183E0253F380710F024EF33E021
:100F4000C901089580914403909145038F5F9F4F9D
:100F5000E9F08091C602482F50E0A4E4B3E020E01D
:100F600030E02417350761F0F8948D919C9111972A
:100F7000F901EE0FFF1FE05AFD4F918380837894B3
:100F80002F5F3F4F12962031310559F70895982F62
:100F90008091BA02873269F4992331F08091B000D0
:100FA00080618093B00008958091B0008F7E80931F
:100FB000B00008951F93CF93DF93EC0170E0CB0155
:100FC0008270907060FF1AC0892B31F080916603A7
:100FD00088831092E40345C01091E40382ED92E00F
:100FE0000E941E011817D8F5E12FF0E0EE55FC4FD6
:100FF000808188831F5F1093E40333C0892BC1F085
:1010000098819093E3031092E403892F807E8036C9
:1010100051F480916603823010F188818F71809342
:10102000250383E01AC09E3FE1F41092660317C0C7
:101030008091E3038F3FA9F42091E403293278F4EF
:10104000E22FF0E0EE52FD4F88818083822F8F5F88
:101050008093E403893229F481E08093660380E081
:1010600001C081E0DF91CF911F910895EF92FF922F
:101070000F931F93CF93DF9380E260E040E02AED6F
:1010800037E00E941B0510926603E2E0EE2E75E049
:10109000F72E04E080916603813039F480E00E94ED
:1010A0001904E09266034398F5CF1091660313305C
:1010B00061F44298809125030E9429031093B6029F
:1010C0000E94F80400936603E5CF809166038430A4
:1010D00009F78091B6028430E9F68FE70E94F402A6
:1010E000C0E0D0E007C00E940803FE01EE55FC4FAF
:1010F0008083219682ED92E00E941E0190E0C81745
:10110000D9078CF3F0926603429AC4CFA0E0B0E016
:10111000ECE8F8E00C94AB20EC010E94FF1A5B01B4
:101120006C017E0100E010E011C0209779F00E9470
:10113000FF1A6A197B098C099D09E616F70608074C
:10114000190720F40E943E0581E008C08091070342
:1011500082FDEBCF8091080310920803CDB7DEB774
:10116000EAE00C94C720A0E0B0E0E9EBF8E00C94D2
:10117000AD20182F7B01042FC22FD0E0F4E0CF2E3A
:10118000D12CCC22DD2222FF03C080E090E004C0FD
:1011900080918002909181020E948608282F8823E6
:1011A000B9F51092080300930603F0920503E0924C
:1011B0000403110F11601093030390910703C1FD05
:1011C00002C084E001C085E0892B809307038091F1
:1011D000070381FF0BC0809107038D7F8093070376
:1011E000809103038093BB0085EC01C085EE809362
:1011F000BC00C0FF0DC0C114D10419F080E090E024
:1012000004C080918002909181020E948608282F5C
:10121000822FCDB7DEB7E8E00C94C920A0E0B0E0A3
:10122000E4E1F9E00C94AD20182F7B01042FC22FCC
:10123000D0E0A4E0CA2ED12CCC22DD2222FF03C0B4
:1012400080E090E004C080918002909181020E9431
:101250008608282F8823B1F510920803009306030F
:10126000F0920503E0920403110F10930303909191
:101270000703C1FD02C084E001C085E0892B809393
:1012800007038091070381FF0BC0809107038D7FC7
:1012900080930703809103038093BB0085EC01C01A
:1012A00085EE8093BC00C0FF0DC0C114D10419F0BD
:1012B00080E090E004C080918002909181020E94C1
:1012C0008608282F822FCDB7DEB7E8E00C94C9201E
:1012D0008091B602813011F081E008950E94FF1ADA
:1012E0002091FD023091FE024091FF0250910003D7
:1012F000621B730B840B950B615A764881409040BA
:1013000010F480E0089582E00895FF920F931F93F8
:10131000CF93DF93182F092FF62E8EE30E941E0322
:10132000212F302FC901EC0110E005C08FE7699132
:101330000E941E031F5F1F15C8F385E064E00E9432
:101340001E0383E00E9418038093FB0284E00E9446
:1013500018038093FC020E94FF1A6093FD027093B1
:10136000FE028093FF029093000387E069E00E94F1
:101370001E0381E08093B602CDB7DEB7E5E00C94A2
:10138000CC200E9485098091B6028130D9F40E9458
:10139000FF1A2091FD023091FE024091FF02509110
:1013A0000003621B730B840B950B605A76488140D7
:1013B000904040F4E8CF8DE794E060E071E00E9457
:1013C000E71D08958091B6028130A9F30895A1E048
:1013D000B0E0EDEEF9E00C94B3208091660382302A
:1013E000B9F480E2BE016F5F7F4F41E021E00E94CF
:1013F000B308882379F08FEF809366030E94F11A77
:1014000060936703709368038093690390936A0302
:101410008FEF01C089812196E2E00C94CF20A1E0FA
:10142000B0E0E5E1FAE00C94B320809166038230ED
:10143000D9F480912503805A898380E2BE016F5FD1
:101440007F4F41E021E00E940E09882369F08FEF71
:10145000809366030E94F11A609367037093680398
:101460008093690390936A032196E2E00C94CF2065
:10147000AAE2B0E0EEE3FAE00C94B1208FEF8983AA
:10148000DE011296E2EDF2E089E201900D928150C8
:10149000E1F780E28E010F5F1F4FB8014AE221E0C1
:1014A0000E940E09882351F480E2B80141E021E056
:1014B0000E94B308882311F482E001C08FEF80936B
:1014C000660380916603823051F00E94F11A6093A6
:1014D0006703709368038093690390936A03AA96E5
:1014E000E4E00C94CD20A2E0B0E0E9E7FAE00C944F
:1014F000AF200E94FF1A9B01AC01809109039091DB
:101500000A03A0910B03B0910C0379018A01E81A38
:10151000F90A0A0B1B0BD801C70181519742A04061
:10152000B04008F444C080910D038F5F80930D0399
:10153000815080FD02C000E001C007E02093090354
:1015400030930A0340930B0350930C038DE794E010
:1015500063E00E949F1F8DE794E061E00E949F1F5F
:1015600047E0F42EF00E802F90E0880F991F9C0129
:10157000205A3D4F3A832983F90160817181672F99
:10158000772763707070880F991F682B792B8DE710
:1015900094E00E949F1FE981FA81608171817070DF
:1015A0008DE794E00E949F1F0F5F0F15E1F62296D2
:1015B000E6E00C94CB201F93182F8DE794E0612F69
:1015C0000E949F1F812F0E94C8001F910895A0E0D4
:1015D000B0E0EDEEFAE00C94AD20082F0E94FF1A67
:1015E0009B01AC018091090390910A03A0910B0328
:1015F000B0910C0369017A01C81AD90AEA0AFB0AF8
:10160000D701C60181519742A040B04008F443C0C1
:101610002093090330930A0340930B0350930C0368
:101620001092E7031092E60388EA0E94DB0A002387
:1016300011F481E001C081E80E94DB0A80E10E9490
:10164000DB0AC0E0D0E0FE01EE0FFF1FE05AFD4FC5
:10165000808191810E9477028C0153E0000F111F5D
:101660005A95E1F7812F0E94DB0A802F0E94DB0A46
:101670002196C031D10539F76091E7038DE794E0F9
:101680000E949F1F6091E6037091E70370708DE7E1
:1016900094E00E949F1FCDB7DEB7E8E00C94C9200C
:1016A000A0E0B0E0E6E5FBE00C94AD20182F062F9B
:1016B0000E94FF1A9B01AC018091090390910A03DB
:1016C000A0910B03B0910C0369017A01C81AD90AE1
:1016D000EA0AFB0AD701C60181519742A040B040F7
:1016E00008F4D6C12093090330930A0340930B03F7
:1016F00050930C038091600290916102880F991FB2
:1017000080930E03977080910F03887F892B8093BD
:101710000F032091620230916302220F331F922F38
:10172000990F990F990F8770892B80930F03422F80
:1017300042954695477080911003807C932F977057
:10174000990F990F990F842B892B80931003209167
:10175000640230916502220F331F922F9295990FE8
:10176000990F907C8F73892B80931003932F929500
:10177000990F990F907C822F86958695892B80935F
:101780001103932F969596959170809112038E7FF9
:10179000892B809312032091660230916702220FF9
:1017A000331F922F990F8170892B80931203422F40
:1017B000441F4427441F80911303807F932F977009
:1017C000990F842B892B8093130320916802309109
:1017D0006902220F331F922F9295907F8F70892B71
:1017E00080931303422F42954F70809114038078A9
:1017F000932F97709295907F842B892B809314035D
:1018000020916A0230916B02220F331F8F778093F1
:101810001403932F979599279795822F8695892B57
:1018200080931503932F96959370809116038C7F68
:10183000892B8093160340916C0250916D02440FE6
:10184000551F942F990F990F8370892B809316033E
:10185000942F929596959695937020911703207EDC
:10186000852F8770880F880F292B282B209317032B
:1018700080916E0290916F02880F991F382F3295D8
:10188000330F307E2F71232B20931703292F22959E
:10189000220F207E869586958695822B809318034D
:1018A0008091700290917102880F991F80931903A3
:1018B000977080911A03887F892B80931A03209157
:1018C000720230917302220F331F922F990F990FDA
:1018D000990F8770892B80931A03422F4295469562
:1018E000477080911B03807C932F9770990F990FFD
:1018F000990F842B892B80931B03209174023091C4
:101900007502220F331F922F9295990F990F907C99
:101910008F73892B80931B03932F9295990F990FA7
:10192000907C822F86958695892B80931C03932F1C
:1019300096959695917080911D038E7F892B80934B
:101940001D032091760230917702220F331F922FD0
:10195000990F8170892B80931D03422F441F4427C8
:10196000441F80911E03807F932F9770990F842BC3
:10197000892B80931E032091780230917902220FE7
:10198000331F922F9295907F8F70892B80931E0327
:10199000422F42954F7080911F038078932F97704C
:1019A0009295907F842B892B80931F0320917A023C
:1019B00030917B02220F331F8F7780931F03932F69
:1019C000979599279795822F8695892B8093200349
:1019D000932F96959370809121038C7F892B809310
:1019E000210340917C0250917D02440F551F942F9A
:1019F000990F990F8370892B80932103942F9295CF
:101A000096959695937020912203207E852F87705E
:101A1000880F880F292B282B2093220380917E0288
:101A200090917F02880F991F382F3295330F307EA7
:101A30002F71232B20932203292F2295220F207E02
:101A4000869586958695822B80932303112311F426
:101A500090E001C098E0002311F480E001C084E030
:101A6000892B809324038DE794E06FE00E949F1FF1
:101A7000CEE0D3E08DE794E069910E949F1F83E060
:101A8000C532D807B9F78DE794E060E00E949F1F48
:101A9000CDB7DEB7E8E00C94C9200F931F93809177
:101AA0003E0390913F039F770E949C02982F8F30B6
:101AB00029F480913A038695805804C089E0989F64
:101AC000C001112480933B030091C602003170F4E1
:101AD000F89410E080913B030E948E07000F111FC5
:101AE000005A1D4FF8019183808378948091BA0247
:101AF0008132C9F490913B03892F81508E3F60F071
:101B00008091B0008F7D8093B00060E0911161E022
:101B100083E00E94FA1B07C09093B4008091B0004C
:101B200080628093B0001F910F9108951F93182F2A
:101B3000811111E082E1612F0E94FA1B83E1612F84
:101B40000E94FA1B10920603109207038091B900BD
:101B50008C6F8093B90080E28093B80085E4809315
:101B6000BC001F910895CF93DF938DE794E00E940E
:101B70002C1F892BF9F08091E103C82FD0E09E0142
:101B80002F5F3F4F2F7130708091E00390E0281756
:101B9000390781F08DE794E00E94661FC054DC4F46
:101BA00088838091E10390E001968F71907080931B
:101BB000E103DBCFDF91CF910895EF92FF921F9366
:101BC000CF93DF9382ED92E00E94280180938402FC
:101BD0009091C602981719F49F5F90938402EDE6E6
:101BE000F3E0108211821282339623E0EF37F2077E
:101BF000C1F78FEF80939D0380939E0380939F0393
:101C0000E8EBEE2EE2E0FE2EACE8B2E0E7016FEF8B
:101C10005FEF4FEF88818031F0F490E03C91FC0160
:101C2000EE0FFF1FE80FF91FE359FC4F8081832B54
:101C3000808311962C9111978181822B818312963A
:101C40009C9112978281892B828330954323209522
:101C50005223909569232196139682E0CE3BD807B4
:101C6000C9F660939F0350939E0340939D03C6E87B
:101C7000D2E010E0F7018081823238F08632B0F095
:101C8000863219F4888160E00FC0143021F480910D
:101C9000C1008F7E05C0153029F48091C100877F77
:101CA0008093C100888161E00E948E1B1F5F0894B1
:101CB000E11CF11C21961630E9F68091B8028032C1
:101CC00031F489E061E00E94FA1B82E801C082E001
:101CD0008093800081E08093410380934203809150
:101CE000BA02813211F08732C9F483E061E00E94C8
:101CF0008E1B83E060E00E94FA1B8091BA02813261
:101D000021F481E08093B00009C082E08093B000AC
:101D100085E08093B1008EE38093B3008AE18093E5
:101D200081008FEF9FEF909389008093880080ED72
:101D300097E0909387008093860080E49CE99093DD
:101D40008302809382029093A1038093A003109258
:101D5000400380916F00816080936F008091C50285
:101D600083FF0DC080914403909145038F5F9F4F87
:101D700031F00E94A2071092420310924103DF91BA
:101D8000CF911F91FF90EF9008958CE060E00E944A
:101D90008E1B8BE061E00E948E1B8DE061E00E9453
:101DA0008E1B82E060E00E948E1B84E061E00E9456
:101DB0008E1B089583E00E9418038093FB0284E049
:101DC0000E9418038093FC0287E061E00E941E03DA
:101DD0006AE070E080E090E00E94251B0E94F80419
:101DE000000008950F931F93082F17C0439A64E6CD
:101DF00070E080E090E00E94251B439864E670E06C
:101E000080E090E00E94251B1F5F101778F36CE2C2
:101E100071E080E090E00E94251B10E0F6CF482F93
:101E2000392F25E00DC0F999FECF1FBA842F932FCB
:101E300092BD81BD60BD0FB6F894FA9AF99A0FBEB3
:101E4000215059F0F999FECF842F932F92BD81BD77
:101E5000F89A80B5681739F7089582E00E94F20E6B
:101E60000895A0E0B0E0E7E3FFE00C94A520482E41
:101E7000562EEE24FF24C0E0D0E0CC24DD248824BC
:101E8000992404C055245394CC24DD24442051F4D7
:101E900087EBE82E82E0F82EC0E0D0E00BE1802E48
:101EA000912C19C021E0421651F412EDE12E12E0FE
:101EB000F12ECDE1D0E0B9E28B2E912C0CC032E0B6
:101EC000431649F4A4E4EA2EA3E0FA2EC8E4D0E0D5
:101ED000F0E28F2E912C3E016C0C7D1C1092E703DA
:101EE0001092E603E3011BC0552059F4F999FECF87
:101EF000D2BDC1BDF89A80B5F701E00FF11F808314
:101F000007C0F701E00FF11FCE0160810E940F0FA3
:101F10000E0D1F1DF80180810E94C80021969E01B0
:101F20002619022F10E008151905F0F2CE015520F0
:101F3000D9F4F999FECFD2BDC1BDF89A20B5F9996F
:101F4000FECF2196D2BDC1BD2197F89A80B590E011
:101F5000B22EAA248A299B292091E6033091E70317
:101F60002817390759F48ECF21966091E7030E9414
:101F70000F0FCE016091E6030E940F0F80E091E009
:101F8000C80ED91E91E0C91693E0D90608F47ECF99
:101F9000852DCDB7DEB7E0E10C94C12082E060E092
:101FA0000E94310F882331F48FEF9FEF9093450308
:101FB00080934403089582E061E00E94310F089508
:101FC00095E09093B70290E29093B80226E22093B6
:101FD000B90291E29093BA022093BB0294E29093EB
:101FE000BC0295E29093BD0292E09093C5029FEFF0
:101FF0009093C6022AE02093CF021092D002109252
:10200000D1021092C7021092C8021092C902109217
:10201000CA029EE19093CB022093CC0228EB3BE0D6
:102020003093CE022093CD02882361F080E061E0FE
:102030000E94310F8FEF9FEF9093450380934403ED
:102040000E94DB0F0895ABE5B0E0E9E2F0E10C940B
:10205000A3205B016C010E94F11A1B012C0181E09D
:102060000E94190483E08093B6020E94DA0E8DE785
:1020700094E06CE071E00E94E71D3E010894611C51
:10208000711CE4C08DE794E06AE171E00E94E71DF5
:102090008FE70E94F4020E940803182F898382367A
:1020A00001F502ED12E00E940803F80181938F010F
:1020B000F2E00B3F1F07B9F78091D202873309F096
:1020C000C0C08DE794E063E271E00E94E71D82E406
:1020D0008983CE01019661E00E94C109429A81E0A4
:1020E000CBC0803719F0893631F506C020E52A8348
:1020F000AA24BB24650105C081E00E94E00F89E4A9
:102100008A838091E503882321F08091C50280684D
:1021100003C08091C5028F778093C502DE011396BC
:10212000E7EBF2E08BE101900D928150E1F7CE01F7
:1021300002966CE184C08437E1F434E53E8F83E09D
:102140008F8F90E798A3E6E0E9A3FCE0FAA3DE0115
:102150009396E6EDF1E088E101900D928150E1F770
:10216000CE014E966DE10E94C109AA24BB246501EF
:1021700068C0853791F407EB12E00E940803F8016C
:1021800081938F01F2E0023D1F07B9F780E061E023
:102190000E94310F25E5298350C0863631F58091A4
:1021A0004403909145038F5F9F4FD1F086E48BAF3E
:1021B00094E4E92E93E0F92E8E01045C1F4FF701A1
:1021C000819191917F010E947702F8019083818330
:1021D0000E5F1F4FF4E6EF16F3E0FF0681F701C034
:1021E0001BAFCE01CB9661E22AC08736D9F404E456
:1021F00013E00E940803982E88240E94080394018B
:10220000280F311DC9010E944802F8018193919362
:102210008F01F3E004361F0761F727E429830E944A
:10222000DB0F0BC0873469F48FEF9FEF909345036A
:10223000809344030E94DB0F1983C30161E00E9475
:10224000C10993E09093B6020E94F804A114B1046E
:10225000C104D10459F00E94F11A6219730984096A
:1022600095096A157B058C059D0528F48091B602B9
:10227000843061F707CF80E0C55ADF4FE2E10C946C
:10228000BF2080E060E00E94310F882319F481E0D4
:102290000E94E00F089581E061E00E94310F0895EF
:1022A00081E060E00E94310F882311F490E006C0C5
:1022B00090E08091D202873309F491E0892F08954C
:1022C000EF92FF920F931F93CF93DF93EB019C014B
:1022D000442737FD4095542F60E271EA87E090E093
:1022E0000E94882089011216130614F001E010E004
:1022F000BE01882777FD8095982F20E231EA47E0DC
:1023000050E00E9433209801442737FD4095542F18
:102310000E9488207901C0E0D0E009C02B9AC80152
:102320000E94491B2B98C8010E94491B2196CE157B
:10233000DF05A4F3CDB7DEB7E6E00C94CB20429ADC
:1023400083E00E9418038093FB0284E00E9418033C
:102350008093FC0286E060E00E941E0387E061E05B
:102360000E941E0389E06FE70E941E038AE065E079
:102370000E941E038BE062E10E941E038CE065E177
:102380000E941E038DE06DEF0E941E038EE060E050
:102390000E941E0380E76CE20E941E0380E360E05F
:1023A0000E941E0389E760E00E941E038AE765E041
:1023B0000E941E0381E762E10E941E0382E762E041
:1023C0000E941E0383E760E00E941E0384E760E032
:1023D0000E941E036091C7027091C8028091C902D9
:1023E0009091CA020E94AF038DE667E00E941E032F
:1023F0006AE070E080E090E00E94251B87E069E0E1
:102400000E941E036AE070E080E090E00E94251BBD
:1024100088E891E061E070E00E946011A8958DE687
:1024200065E00E941E036AE070E080E090E00E9498
:10243000251B88EB91E061E070E00E946011A89597
:102440008DE664E00E941E036AE070E080E090E0A8
:102450000E94251B8DE591E061E070E00E94601113
:10246000A8958DE662E00E941E036AE070E080E0BD
:1024700090E00E94251B8FEA90E061E070E00E94EE
:102480006011A8958DE660E00E941E036AE070E08E
:1024900080E090E00E94251B85E091E062E070E022
:1024A0000E946011A89587E061E00E941E03429897
:1024B0000895A6E1B0E0EFE5F2E10C94A520A8951F
:1024C0008CE00E941803882359F48DE794E06EE2B3
:1024D00071E00E94E71D80E00E9419040E94DA0E5C
:1024E0000E94B30D0E94FF1A0E94E709B82E8E01C8
:1024F0000F5F1F4FAA24AA948091B602843029F05E
:1025000045E0E42EBE1409F096C10E94FF1A6B014B
:102510007C018091B6028430E9F48FE70E94F402D6
:1025200000E010E008C00E940803F801EE55FC4FDF
:1025300080830F5F1F4F82ED92E00E941E0190E0AA
:102540000817190784F30E94430390933D03809377
:102550003C0328C082ED92E00E941E01482F4F5F8D
:1025600080E2B80121E00E94B308882369F0A092BC
:1025700066030E94F11A6093670370936803809367
:10258000690390936A03B8CF82ED92E00E941E0126
:10259000482F22EA33E0FE013296C901BF0150E024
:1025A0000E948C00C0922603D0922703E092280359
:1025B000F09229031092650380913E0390913F03AE
:1025C000880F991F816090933F0380933E03439847
:1025D000429A80E00E94C7078091A203282F30E032
:1025E000C9018E739070892B09F041C0F8948091D5
:1025F000FA02877060E672E043EA53E00E94AC01A1
:102600000091C602003160F410E080913B030E940B
:102610008E07000F111F005A1D4FF8019183808310
:1026200078948091A20390916C0380FF1BC0992342
:1026300009F045C0A4E4B3E020E030E0F901EE0F7A
:10264000FF1FE05AFD4F808191818D939D932F5FF5
:102650003F4F2031310591F70E94DB0F81E08093DD
:102660006C032DC0992359F110926C0328C0C90145
:1026700088739070C89719F54091B703842F82270B
:1026800087FF1DC040584093B7038091BD0285323B
:10269000B1F410E00AC01F5FE12FF0E0EE55FC4FEF
:1026A0008DE794E060810E949F1F212F30E0809190
:1026B000A20390E0877090708217930764F780916F
:1026C0006403882319F481E0809364031092430328
:1026D00010924103109242038091FA02887109F42A
:1026E000A1C04091B7038091A20390E0242F30E075
:1026F0008227932786FD60C0407C80E44827409372
:10270000B7039091E0038091E103981701F1A8EBE2
:10271000B3E030E00FC03F5F892F90E0FC01E05450
:10272000FC4F20812D9301968F7190708093E00370
:10273000383031F09091E0038091E103981759F718
:10274000395C8091B703382B3093B70335C0809143
:1027500039038093B8038091B902863251F482E143
:102760000E945D1C95958795959587958093B903F3
:1027700002C01092B9038091BB02863251F483E10A
:102780000E945D1C95958795959587958093BA03D2
:1027900002C01092BA0380913D038093BB038091E5
:1027A0003C038093BC0380913E0390913F039F774D
:1027B0000E949C028093BD0387EB93E069E00E9436
:1027C000850902C00E94B30D0E9468098823D1F3D5
:1027D00008EB12E056E8E52E52E0F52EF801808174
:1027E000E82FF0E0CF01807F9070409791F4EF7078
:1027F000F070EE0FFF1FE05AFD4F8081918160E085
:102800008F3F910511F008F061E0F70180810E948F
:10281000FA1B0F5F1F4F0894E11CF11CF2E00E3B06
:102820001F07E1F683E08093B6020E94F80481E07E
:1028300080936B0342980E94FF1A5B016C010E9417
:10284000F11A2B013C0180916503823008F065C0CC
:10285000E0902603F09027030091280310912903AC
:1028600080912A0390912B03A0912C03B0912D030A
:102870008E159F05A007B10709F44FC082ED92E0C5
:102880000E943801A60195012E193F09400B510BFA
:102890006C5D754080409040621773078407950710
:1028A000E0F5E0922A03F0922B0300932C0310939F
:1028B0002D030E943F038093390320913703309109
:1028C0003803280F311D309338032093370360916C
:1028D00036036F5F609336036930F8F0C90170E02A
:1028E0000E945220CB0170933803609337032091EC
:1028F0003A0343E0249F90011124820F931F969581
:1029000087959695879580933A030E944D0D109276
:10291000380310923703109236038091640390902D
:10292000E203882309F457C180906503891408F0F5
:10293000D5C182ED92E00E943801209126033091AA
:1029400027034091280350912903A21AB30AC40A0D
:10295000D50A68517C4F8F4F9F4F6A157B058C05B8
:102960009D0508F075C080913E0390913F03880F4C
:10297000991F90933F0380933E0381E080936B0304
:10298000882081F440922E0350922F0360923003EE
:102990007092310310923203109233031092340379
:1029A00010923503809165038F5F8093650382EDFC
:1029B00092E00E9438012091260330912703409134
:1029C000280350912903260F371F481F591F2093B2
:1029D000260330932703409328035093290381E073
:1029E00080936B03439A0E94C7070E944D0D30C02D
:1029F00082ED92E00E9438019B01AC018091260398
:102A000090912703A0912803B091290386017501B5
:102A1000E81AF90A0A0B1B0B682D70E080E090E0C1
:102A20000E9433206E157F058007910788F410926D
:102A30003F0310923E0381E080936B030E944D0D93
:102A4000A0922603B0922703C0922803D0922903B4
:102A500080916503882309F4E8C09091CF029923FF
:102A600089F180914303882369F5892F90E00E94C2
:102A7000E50020912E0330912F03409130035091B7
:102A8000310383017201E21AF30A040B150B6E1570
:102A90007F0580079107B0F481E0809343030E9493
:102AA000A2078091CB020E941801640D751D861D3E
:102AB000971D6160609332037093330380933403F6
:102AC000909335039091D1029923F1F080914103C5
:102AD0008823D1F4892F90E00E94E50020912E03F5
:102AE00030912F03409130035091310383017201E3
:102AF000E21AF30A040B150B6E157F058007910788
:102B000018F481E0809341039091D0029923F1F071
:102B1000809142038823D1F4892F90E00E94E50040
:102B200020912E0330912F034091300350913103B7
:102B300083017201E21AF30A040B150B6E157F056F
:102B40008007910718F481E0809342038091C702C7
:102B50009091C802A091C902B091CA020097A10544
:102B6000B10509F462C08091320390913303A091C2
:102B70003403B09135030097A105B10509F455C0A0
:102B800083017201E81AF90A0A0B1B0B17FD4DC0ED
:102B90006091CC0270E080E090E028EE33E040E00D
:102BA00050E00E9433206E157F0580079107E8F5FD
:102BB0000E949F1180E00E9419040E94F8040E9464
:102BC000F11A61606093320370933303809334038E
:102BD000909335032AC082ED92E00E9438019B0158
:102BE000AC018091260390912703A0912803B09116
:102BF000290386017501E81AF90A0A0B1B0B692DD6
:102C000070E080E090E00E9433206E157F05800721
:102C1000910758F4A0922603B0922703C09228038C
:102C2000D092290381E080936B0380914203882333
:102C3000B1F48091BD02883219F40E94730A0FC06A
:102C4000893239F480914303609165030E94500BEF
:102C500006C08A3221F4809143030E94E70A8091E2
:102C60006B038823B9F0E0912503EF5FE093250320
:102C7000E83131F0F0E0EE52FD4F8785882311F402
:102C800010922503809125030E9429030E940F0AB8
:102C900010926B03809166038F3F21F50E94F11A19
:102CA00020916703309168034091690350916A0352
:102CB000621B730B840B950B695E734080409040E0
:102CC00088F00E94F11A6093670370936803809301
:102CD000690390936A030E94380A04C0891409F0BA
:102CE000B7CE86CE6696E0E10C94C120FF920F939A
:102CF0001F93082FF62E61E00E948E1B802F61E04B
:102D00000E94FA1B8F2D61E00E94FA1B8AE090E07E
:102D10000E94491B8F2D0E942D1C892B11F410E05D
:102D20000FC0802F60E00E94FA1B8AE090E00E94B2
:102D3000491B8F2D0E942D1C10E0892B09F411E0F6
:102D4000802F60E00E948E1B802F60E00E94FA1BA3
:102D50008F2D60E00E94FA1B812F1F910F91FF9031
:102D60000895EF92FF920F931F938C016DE7E62E6B
:102D700064E0F62EC701612F70E04AE050E00E9447
:102D8000641DC7016EE20E94A31C54E016950795CE
:102D90005A95E1F70F701070C701B8014AE050E092
:102DA0000E94641D1F910F91FF90EF900895A2E281
:102DB000B0E0EDEDF6E10C94A3208E010F5F1F4F04
:102DC00080E1D8011D928A95E9F78DE794E066E3EA
:102DD00071E00E94E71D0E94DA0E20EC3DE948E513
:102DE00055E32F8F38A349A35AA380EC97EFAAEBA2
:102DF000B7E38B8F9C8FAD8FBE8F24EF31E040E027
:102E000050E02F8B388F498F5A8FA0E5CA2EA3EC44
:102E1000DA2EE12CF12CF0EC4F2EFDE95F2EF8E5D7
:102E20006F2EF5E37F2E88249924540133241E8AC3
:102E30001D8A198A1A8A1B8A1C8AFFC08DE794E0B2
:102E40000E94661F8434B9F0853430F48332B9F1BE
:102E50008C3209F0CCC044C0833509F0C8C02F8D36
:102E600038A149A15AA1C901DA012C013D018824E8
:102E700099245401E2C08DE794E064E40E94A31C0D
:102E80008DE794E040EC5DE968E575E32AE030E029
:102E90000E94871D8DE794E06CE20E94A31C8DE7E1
:102EA00094E040EC57EF6AEB77E32AE030E00E94D1
:102EB000871D8DE794E06CE20E94C11CBEC01982A0
:102EC0001A821B821C821D821E821F82188619860E
:102ED0001A861B861C861D861E861F86188A3AC087
:102EE000339434E0331609F0A8C069817A818B816C
:102EF0009C8128EE33E040E050E00E9433206F8F49
:102F000078A389A39AA36D817E818F8198850E9481
:102F100033206B8F7C8F8D8F9E8F89859A85AB85B3
:102F2000BC858F8B988FA98FBA8F6D857E858F8595
:102F300098890E9433206B017C0190E2C9169EE4BF
:102F4000D90690E0E90690E0F90630F48CE162E3FE
:102F50000E941E03332471C0A0E3CA16A5E7DA0657
:102F6000A0E0EA06A0E0FA0618F48CE162E2F0CFF5
:102F7000B0E4CB16BCE9DB06B0E0EB06B0E0FB0644
:102F800018F48CE166E2E4CFE0E5CE16E3ECDE0671
:102F9000E0E0EE06E0E0FE0618F48CE162E1D8CF56
:102FA000F0E6CF16FAEEDF06F0E0EF06F0E0FF06FF
:102FB00018F48CE165E1CCCF20E7C21621E1D206FE
:102FC00021E0E20620E0F20618F48CE161E0C0CFD7
:102FD00030EAC31636E8D30631E0E30630E0F30604
:102FE00018F48CE163E0B4CF8CE165E0B1CFE0EDA3
:102FF0002E2E280E49E0421500F1032D10E0000F9F
:10300000111F000F111F81E090E08C0F9D1F080F12
:10301000191FD8016D917D918D919C912AE030E02E
:1030200040E050E00E943320620D711D811D911D12
:10303000F80160837183828393838DE794E00E941B
:103040002C1F892B09F0FACE81149104A104B1043C
:1030500089F4C301B2010E94AF0361E070E080E037
:1030600090E00E94251BFFEFFE8B1D8A198A1A8AA9
:103070001B8A1C8A2F89388D498D5A8D821693069A
:10308000A406B506E0F40E943F0329893A894B89DA
:103090005C89280F311D411D511D298B3A8B4B8BAB
:1030A0005C8B3D89381708F48D8B4E89841708F4A2
:1030B0008E8B0894811C911CA11CB11C56C0C301AD
:1030C000B20128EE33E040E050E00E9466208DE738
:1030D00094E0BA01A9012AE030E00E94551D8DE775
:1030E00094E06CE20E94A31C8DE794E06D894AE0B5
:1030F00050E00E94751D8DE794E06CE20E94A31CD5
:1031000069897A898B899C89A50194010E9466202E
:103110008DE794E0BA01A9012AE030E00E94551D34
:103120008DE794E06CE20E94A31C8DE794E06E8929
:103130004AE050E00E94751D8DE794E06CE20E9429
:10314000C11C4C0C5D1C6E1C7F1C8B8D9C8DAD8D31
:10315000BE8D84159505A605B70520F44F8C58A0A3
:1031600069A07AA08824992454012F8D38A149A1FF
:103170005AA1285E33404040504009F05ECFA296ED
:10318000E2E10C94BF2080E065E970E042E050E0AD
:103190000E942C1A0895A1E0B0E0E1EDF8E10C9452
:1031A000B32080E00E94B10080E161E00E948E1BAC
:1031B00081E161E00E948E1B0E94C50E80E060E00C
:1031C0000E948E1B81E061E00E948E1B8DE794E0DF
:1031D00040E052EC61E070E00E94A51E0E944111A7
:1031E0000E94CE0F8DE794E063E471E00E94E41D3D
:1031F00080E793E00E94B1168DE794E06AE571E004
:103200000E94E41D8DE794E068E070E04AE050E041
:103210000E94D01D0E94C3187894439A83E063E112
:103220000E947616882329F0439842980E94D71668
:10323000FBCF89E062E10E947616882329F40E9480
:103240005011882309F000C18DE794E062E671E037
:103250000E94E41D60E070E080E090E00E94231096
:10326000882349F00E944B118DE794E06BE971E0EF
:103270000E94E71D429A0E94DD0D22C08091BB0290
:10328000833229F08091C5028B7F8093C5028091A3
:10329000C50281FF15C082FD13C064EF71E080E0BC
:1032A00090E00E942310882359F00E944B118DE773
:1032B00094E06BE971E00E94E71D0E94DD0D429AE7
:1032C0008091B902823239F58091BB02833219F5BF
:1032D00081E00E94960D8091C50282FF09C08DE7B2
:1032E00094E066EB71E00E94E71D0E94360813C06F
:1032F00064E170E080E090E00E94251B80E2BE0166
:103300006F5F7F4F41E021E00E94B308882319F4EA
:1033100081E0809366038DE794E061EC71E00E94A8
:10332000E41D8FE00E94B10080E00E941904109219
:10333000250380E00E9429031092E20390E0983177
:1033400058F4292F2F5FE92FF0E0EE52FD4F8785CB
:10335000882311F0922FF3CF9093E20383E08093C0
:10336000B6020E94DA0E80916603882311F00E9453
:10337000380A8091BD02883211F08A3239F48DE723
:1033800094E040E052EC61E070E02BC0893271F4CF
:103390008DE794E040EA56E861E070E00E94A51EE7
:1033A0008091C20080628093C20022C08091FA02A4
:1033B0008871803169F04091D3025091D4026091BC
:1033C000D5027091D6024A3051056105710538F475
:1033D0008DE794E040E855E260E070E002C08DE7E0
:1033E00094E00E94A51E04C08DE794E00E94661F31
:1033F0008DE794E00E942C1F892BB1F78091BC02CD
:10340000843229F08091C1008F7E8093C100809129
:10341000BD02853229F08091C100877F8093C10071
:103420001092E0031092E103109264030E94FF1ACD
:1034300060932603709327038093280390932903B6
:103440002196E2E00C94CF200E94DD0D8091B9021C
:10345000823209F017CF12CF823000F5E82FF0E06A
:10346000EE0FFF1FE851FC4F71836083882319F032
:103470008130A1F408C0809169008C7F842B8093F7
:103480006900E89A089580916900440F551F440F20
:10349000551F837F842B80936900E99A08951F92BA
:1034A0000F920FB60F9211242F933F934F935F9378
:1034B0006F937F938F939F93AF93BF93EF93FF93FC
:1034C0008091E8039091E903892B29F0E091E803CA
:1034D000F091E9030995FF91EF91BF91AF919F9111
:1034E0008F917F916F915F914F913F912F910F90AD
:1034F0000FBE0F901F9018951F920F920FB60F924C
:1035000011242F933F934F935F936F937F938F93E8
:103510009F93AF93BF93EF93FF938091EA039091B2
:10352000EB03892B29F0E091EA03F091EB03099575
:10353000FF91EF91BF91AF919F918F917F916F918B
:103540005F914F913F912F910F900FBE0F901F9061
:1035500018951F920F920FB60F9211242F933F933D
:103560008F939F93AF93BF938091F0039091F1035A
:10357000A091F203B091F3033091F4030196A11DE1
:10358000B11D232F2D5F2D3720F02D570196A11D42
:10359000B11D2093F4038093F0039093F103A09363
:1035A000F203B093F3038091EC039091ED03A091AB
:1035B000EE03B091EF030196A11DB11D8093EC03C2
:1035C0009093ED03A093EE03B093EF03BF91AF91FF
:1035D0009F918F913F912F910F900FBE0F901F9051
:1035E00018958FB7F8942091F0033091F103409132
:1035F000F2035091F3038FBFB901CA0108959FB739
:10360000F8942091EC033091ED034091EE0350913A
:10361000EF0386B5A89B06C08F3F21F02F5F3F4F79
:103620004F4F5F4F9FBF542F432F322F2227280F1A
:10363000311D411D511D82E0220F331F441F551FB4
:103640008A95D1F7B901CA010895EF92FF920F93BD
:103650001F93CF93DF937B018C010E94FF1AEB0134
:103660000EC00E94FF1A6C1B7D0B685E7340C8F38E
:103670000894E108F10801091109C851DC4FE1146F
:10368000F1040105110569F7CDB7DEB7E6E00C944A
:10369000CB20019739F0880F991F880F991F029747
:1036A0000197F1F70895789484B5826084BD84B55C
:1036B000816084BD85B5826085BD85B5816085BD2D
:1036C000EEE6F0E0808181608083E1E8F0E0108246
:1036D000808182608083808181608083E0E8F0E087
:1036E000808181608083E1EBF0E080818460808371
:1036F000E0EBF0E0808181608083EAE7F0E08081A8
:103700008460808380818260808380818160808307
:103710008081806880831092C1000895CF93DF93E9
:10372000482F50E0CA0186569F4FFC0134914A57FA
:103730005F4FFA018491882369F190E0880F991F07
:10374000FC01E859FF4FA591B491FC01EE58FF4FE1
:10375000C591D491662351F42FB7F8948C91932F8F
:10376000909589238C93888189230BC0623061F402
:103770002FB7F8948C91932F909589238C938881FF
:10378000832B88832FBF06C09FB7F8948C91832B1F
:103790008C939FBFDF91CF910895833071F0843077
:1037A00028F48130A1F0823021F514C08630B1F0C8
:1037B0008730D1F08430E9F404C0809180008F77A5
:1037C00003C0809180008F7D80938000089584B530
:1037D0008F7702C084B58F7D84BD08958091B0003D
:1037E0008F778093B00008958091B0008F7D809393
:1037F000B0000895FF920F931F93F62E482F50E0CC
:10380000CA0182559F4FFC012491CA0186569F4FE1
:10381000FC0114914A575F4FFA0104910023C9F04B
:10382000222319F0822F0E94CD1BE02FF0E0EE0F33
:10383000FF1FEE58FF4FA591B4919FB7F894FF205A
:1038400021F48C911095812302C08C91812B8C9353
:103850009FBF1F910F91FF9008950F931F93482FC3
:1038600050E0CA0182559F4FFC012491CA0186563F
:103870009F4FFC0104914A575F4FFA0114911123A5
:1038800019F420E030E015C0222319F0822F0E94A5
:10389000CD1B812F90E0880F991F84589F4FFC010A
:1038A000A591B4918C9120E030E0802311F021E0CB
:1038B00030E0C9011F910F910895982F8E3008F0C4
:1038C0009E509770809185028295880F880F807C2A
:1038D000892B80937C0080917A00806480937A00A9
:1038E00080917A0086FDFCCF20917800409179008C
:1038F000942F80E030E0282B392BC9010895A0E0F7
:10390000B0E0E5E8FCE10C94AD207C016B018A019C
:10391000C0E0D0E00FC0D6016D916D01D701ED91EF
:10392000FC910190F081E02DC7010995C80FD91FC6
:10393000015010400115110571F7CE01CDB7DEB76A
:10394000E8E00C94C920DC01ED91FC910190F0813C
:10395000E02D09950895EF92FF920F931F938C012C
:103960006DE00E94A31C7C01C8016AE00E94A31CB8
:103970009C012E0D3F1DC9011F910F91FF90EF90EB
:103980000895EF92FF920F931F937C010E94A31C56
:103990008C01C7010E94AB1C9C01200F311FC90183
:1039A0001F910F91FF90EF900895CF93DF93EC015B
:1039B0006115710519F420E030E00FC0DB010D90B6
:1039C0000020E9F71197A61BB70BE881F981028067
:1039D000F381E02DAD0109959C01C901DF91CF91E3
:1039E00008954F925F927F928F929F92AF92BF9273
:1039F000CF92DF92EF92FF920F931F93DF93CF93BB
:103A0000CDB7DEB7A1970FB6F894DEBF0FBECDBF1E
:103A10002C01742ECB01223008F42AE019A231E2E5
:103A2000C32ED12CCC0EDD1E822E9924AA24BB24B9
:103A3000672D752FA50194010E94662079018A01E6
:103A4000C801B701A50194010E943320472D461BF0
:103A50000894C108D1084A3010F4405D01C0495CA7
:103A6000F6014083E114F1040105110521F07E2CDB
:103A70005F2DC801DDCFC201B6010E94D51CA19601
:103A80000FB6F894DEBF0FBECDBFCF91DF911F916F
:103A90000F91FF90EF90DF90CF90BF90AF909F90ED
:103AA0008F907F905F904F900895DC012115310534
:103AB00041F4ED91FC910190F081E02D642F099586
:103AC00008950E94F11C0895EF92FF920F931F93A7
:103AD0009A017B0100E010E0B801A7010E94551D8A
:103AE0001F910F91FF90EF900895EF92FF920F9327
:103AF0001F939A01E62EFF2400E010E0B801A70111
:103B00000E94551D1F910F91FF90EF900895A0E026
:103B1000B0E0EDE8FDE10C94AD20EC016A017B0121
:103B20002115310541F4E881F9810190F081E02D02
:103B3000642F09951BC02A303105B1F477FF13C0FB
:103B40006DE20E94A31C8C0144275527BA014C1931
:103B50005D096E097F09CE012AE00E94F11C9C01DB
:103B6000200F311F04C02AE00E94F11C9C01C901F2
:103B7000CDB7DEB7E8E00C94C920EF92FF920F9327
:103B80001F937B019A010027F7FC0095102FB801C5
:103B9000A7010E94871D1F910F91FF90EF9008953C
:103BA000EF92FF920F931F937C010E94BD1D8C0129
:103BB000C7010E94AB1C9C01200F311FC9011F913E
:103BC0000F91FF90EF9008950E94D51C0895EF92F9
:103BD000FF920F931F937C010E94E41D8C01C7018B
:103BE0000E94AB1C9C01200F311FC9011F910F9136
:103BF000FF90EF90089508951F920F920FB60F92C5
:103C000011242F933F934F938F939F93EF93FF93A1
:103C10008091C00082FD1DC04091C60020913504F6
:103C2000309136042F5F3F4F2F73307080913704EF
:103C3000909138042817390771F0E0913504F0911C
:103C40003604EB50FC4F4083309336042093350408
:103C500002C08091C600FF91EF919F918F914F918B
:103C60003F912F910F900FBE0F901F9018951F92AC
:103C70000F920FB60F9211242F933F938F939F9320
:103C8000EF93FF932091790430917A0480917B0423
:103C900090917C042817390731F48091C1008F7D01
:103CA0008093C10014C0E0917B04F0917C04E75C38
:103CB000FB4F208180917B0490917C0401968F734F
:103CC000907090937C0480937B042093C600FF91B6
:103CD000EF919F918F913F912F910F900FBE0F9079
:103CE0001F901895A0E0B0E0E8E7FEE10C94A92051
:103CF000FC011382128288EE93E0A0E0B0E084839E
:103D00009583A683B7838AEA92E09183808375873F
:103D1000648757874687318B208B138B028BF58AFC
:103D2000E48AD78AC68AB18EA08E938E828E8F85C2
:103D3000848F8889858F8989868F8A89878F8B89E7
:103D400080A32096ECE00C94C520AF92BF92DF9246
:103D5000EF92FF920F931F93CF93DF93EC017A01C1
:103D60008B01DD24403081EE580780E0680780E059
:103D7000780711F0DD24D39491E0A92EB12CEC89C1
:103D8000FD89DD2069F0C50108A002C0880F991FD8
:103D90000A94E2F7808360E079E08DE390E005C06B
:103DA000108260E874E88EE190E0A80197010E941B
:103DB00066202150304040405040569547953795F9
:103DC000279580E12030380720F0DD2011F0DD2438
:103DD000D6CFE889F9893083EA89FB89208319A243
:103DE000EE89FF89408121E030E0C9010C8C02C0DE
:103DF000880F991F0A94E2F7482B4083EE89FF89C8
:103E00004081C9010D8C02C0880F991F0A94E2F706
:103E1000482B4083EE89FF894081C9010E8C02C086
:103E2000880F991F0A94E2F7482B4083EE89FF8997
:103E300080810F8C02C0220F331F0A94E2F7209575
:103E400028232083DF91CF911F910F91FF90EF9056
:103E5000DF90BF90AF900895DC011C96ED91FC912E
:103E60001D97E05CFF4F2191319180819181281B4A
:103E7000390B2F733070C90108958DE794E00E94CB
:103E80002C1F892B11F00E94FB1D0895DC011C964C
:103E9000ED91FC911D97E05CFF4F20813181E05452
:103EA000F040DF01AE5BBF4F8D919C9111972817B9
:103EB000390719F42FEF3FEF07C08D919C91E80F60
:103EC000F91F8081282F30E0C9010895DC011C967C
:103ED000ED91FC911D97E05CFF4F20813181E05412
:103EE000F040DF01AE5BBF4F8D919C911197281779
:103EF000390719F42FEF3FEF10C08D919C91119766
:103F0000E80FF91F20818D919C91119701968F7375
:103F1000907011969C938E9330E0C9010895DC0156
:103F200091968C919197882339F05496ED91FC915C
:103F30005597808186FFF9CF91961C920895CF9373
:103F4000DF93EC01EE85FF85E05CFF4F208131813E
:103F5000E054F0402F5F3F4F2F733070DF01AE5BB6
:103F6000BF4F8D919C91119728173907D1F3E05CD1
:103F7000FF4F80819181E054F040E80FF91F60838A
:103F8000EE85FF85E05CFF4F31832083EE89FF895A
:103F9000208181E090E00F8C02C0880F991F0A9465
:103FA000E2F7282B208381E089A3EC89FD898081B9
:103FB0008064808381E090E0DF91CF9108958F92BB
:103FC0009F92AF92BF92CF92DF92EF92FF920F93A8
:103FD0001F9300D000D00F92EDB7FEB7319684E06A
:103FE000ADB7BEB711968C9383E0818387E082835F
:103FF00085E0838381E084838DE794E065EF73E05F
:1040000049E354E025EC30E004EC10E0B0ECEB2E9A
:10401000F12CA1ECCA2ED12CF2ECAF2EB12CE6EC97
:104020008E2E912C0E94721E0F900F900F900F9069
:104030000F901F910F91FF90EF90DF90CF90BF9066
:10404000AF909F908F900895CF93DF930E94531B62
:104050000E94CB18CDE3DFE10E9459122097E1F3D3
:104060000E943D1FF9CF629FD001739FF001829F94
:10407000E00DF11D649FE00DF11D929FF00D839FF7
:10408000F00D749FF00D659FF00D9927729FB00D94
:10409000E11DF91F639FB00DE11DF91FBD01CF01A7
:1040A00011240895AA1BBB1B51E107C0AA1FBB1F07
:1040B000A617B70710F0A61BB70B881F991F5A95B4
:1040C000A9F780959095BC01CD010895A1E21A2E23
:1040D000AA1BBB1BFD010DC0AA1FBB1FEE1FFF1FAC
:1040E000A217B307E407F50720F0A21BB30BE40BFC
:1040F000F50B661F771F881F991F1A9469F7609543
:104100007095809590959B01AC01BD01CF010895FC
:1041100097FB092E05260ED057FD04D0D7DF0AD015
:10412000001C38F450954095309521953F4F4F4FE6
:104130005F4F0895F6F790958095709561957F4F44
:104140008F4F9F4F08952F923F924F925F926F92A1
:104150007F928F929F92AF92BF92CF92DF92EF9217
:10416000FF920F931F93CF93DF93CDB7DEB7CA1B98
:10417000DB0B0FB6F894DEBF0FBECDBF09942A88C3
:10418000398848885F846E847D848C849B84AA846B
:10419000B984C884DF80EE80FD800C811B81AA81F8
:1041A000B981CE0FD11D0FB6F894DEBF0FBECDBFC3
:1041B000ED010895EE0FFF1F0590F491E02D099495
:0441C000F894FFCFA1
:1041C40054582074696D656F757421005761697462
:1041D400696E672062696E640A00476F7420706BB1
:1041E400740A006461746120676F6F640A00525836
:1041F4002068616E67007363616E6E6572206D6F17
:104204006465004F70656E4C52536E67205258209F
:104214007374617274696E672000206F6E20485752
:104224002000454550524F4D2064617461206E6FEB
:10423400742076616C6964206F722062696E6420F8
:104244006A756D70706572207365742C20666F7268
:1042540063696E672062696E640A005361766564FF
:104264002062696E64206461746120746F20454526
:1042740050524F4D0A004920616D20736C61766580
:1042840000456E746572696E67206E6F726D616C45
:10429400206D6F646500002001220126022102279F
:1042A400032303260424052505280529052AC0120D
:1042B40000001A400AA1204EA5001B1E27522C23E1
:1042C400308025000005400AA1204EA50020244E80
:1042D400A52C2330004B000006400AD0009D490065
:1042E4007B289D492C233000E1000005400A45014C
:1042F400D7DC03B81E0EBF00232E48E801008A4015
:104304000A6001555502AD1E20000023C880250017
:104314000005400AA1204EA50020244EA52C2330E0
:104324000002000200020002000200020002000279
:104334000002000200020002000200020002000269
:104344008813409C080109120313000102000000B5
:104354001000000008002000000001000002000717
:104364000B0C10111500000000009F1F7F1C2C1F58
:06437400661F461F8F1FAB
:107E00000F92CDB7DEB7112484B714BE81FFF1D035
:107E100082E08093C00088E18093C10086E0809377
:107E2000C20080E18093C4008EE0CDD088249924E4
:107E3000CC24C394F5E0DF2EE1E1EE2E73E0F72EC3
:107E4000B6D0082F813479F4B2D08983C2D0898129
:107E5000823811F481E005C0813811F485E001C059
:107E600083E09ED09AC0823411F484E103C085344B
:107E700019F485E0B6D091C0853561F498D0082F0B
:107E800010E095D090E0982E8824802A912A880CC2
:107E9000991C82C0863521F484E0A3D080E0E1CF34
:107EA000843609F04CC083D082D0A82E80D0B82E62
:107EB00000E011E07CD0F80181938F01AE16D1F77C
:107EC00088D0FB2DF53489F4E0E0F1E00BC0F9999E
:107ED000FECF92BC81BC0894811C911C819180BD15
:107EE000FA9AF99AEA1598F358C08B2D863409F05E
:107EF00054C0F401F7BEE89507B600FCFDCFF401CD
:107F0000A0E0B1E02C9130E011968C91119790E0B7
:107F1000982F8827822B932B12960C01C7BEE895C9
:107F20001124329681E0A038B80761F7F401D7BE7A
:107F3000E89507B600FCFDCFE7BEE8952EC0843774
:107F4000F1F435D034D0182F32D0B82E42D0FB2DDA
:107F5000F63421F4F40105914F010CC0FB2DF534EA
:107F600049F4F999FECF92BC81BC0894811C911C04
:107F7000F89A00B5802F14D0115049F70EC08537FC
:107F800039F427D08EE10CD085E90AD08FE069CF93
:107F9000813511F488E017D01CD080E101D050CF9A
:107FA0009091C00095FFFCCF8093C600089580910A
:107FB000C00087FFFCCF8091C00084FD01C0A89560
:107FC0008091C6000895E0E6F0E098E19083808318
:107FD0000895EDDF803219F088E0F5DFFFCF84E10E
:107FE000DFCF1F93182FE3DF1150E9F7F2DF1F9166
:0E7FF0000895282E80E0E7DFEE27FF27099492
:027FFE0001057B
:0400000300007E007B
:00000001FF
